:1000000012C02CC02BC02AC029C028C027C026C0BF
:1000100025C024C023C022C021C020C01FC01EC0D4
:100020001DC01CC01BC011241FBECFE5D4E0DEBF25
:10003000CDBF10E0A0E6B0E0EAEAF4E002C005902F
:100040000D92A036B107D9F710E0A0E6B0E001C0EC
:100050001D92A036B107E1F79AD025C2D1CF20ED8D
:1000600037E004C0F9013197F1F701971816190626
:10007000CCF308955D9BFECF8CB980E090E00895AD
:10008000FC0104C05D9BFECF8CB931968081882332
:10009000C9F708955D9BFECF8CB908955F9BFECF95
:1000A0008CB1089587B93F983E9882E886B9309818
:1000B000369A3699FECF84B195B1369A3699FECFED
:1000C00024B135B13798C90108956F927F928F920C
:1000D0009F92AF92BF92DF92EF92FF920F931F9386
:1000E000D82EE0DF3C018D2DDDDF7C018D2DDADFA8
:1000F0004C018D2DD7DF5C018D2DD4DFE60CF71C74
:10010000E80CF91CEA0CFB1CE80EF91E0027F7FCB2
:100110000095102FC801B70126D120E030E040EA59
:1001200050E486D0EDD0CB011F910F91FF90EF905E
:10013000DF90BF90AF909F908F907F906F900895C9
:100140000F931F93DF93CF93CDB7DEB72A970FB6E8
:10015000F894DEBF0FBECDBF8E010F5F1F4FB801F9
:100160004AE050E036D0F80104C05D9BFECF8CB968
:10017000319680818823C9F72A960FB6F894DEBF9E
:100180000FBECDBFCF91DF911F910F9108951F93A7
:10019000CF93DF93539A80B5866880BD549A10BC84
:1001A0008FEC89B980E284BBAD981BE3AD9A5F9B6D
:1001B000FECF8CB1C0E0D0E080E090E086DFC0DF11
:1001C0005D9BFECF1CB9219683E0C032D807A1F712
:1001D000EDCFFB019F01E8944230BCF04532ACF416
:1001E0004A3029F497FB1EF4909581959F4F642F18
:1001F000772745D1805D8A330CF0895D8193CB01EF
:100200000097A9F716F45DE251931082C90100C06E
:10021000DC01FC01672F71917723E1F7329704C06D
:100220007C916D9370836291AE17BF07C8F30895F8
:100230000CD0EBC0E3D040F0DAD030F021F45F3FD7
:1002400019F0CCC0511115C1CFC0F0D098F399234B
:10025000C9F35523B1F3951B550BBB27AA2762178A
:100260007307840738F09F5F5F4F220F331F441FCF
:10027000AA1FA9F333D00E2E3AF0E0E830D0915007
:100280005040E695001CCAF729D0FE2F27D0660FF4
:10029000771F881FBB1F261737074807AB07B0E833
:1002A00009F0BB0B802DBF01FF2793585F4F2AF049
:1002B0009E3F510568F092C0DCC05F3FECF3983E72
:1002C000DCF3869577956795B795F7959F5FC9F7A6
:1002D000880F911D9695879597F90895E1E0660F2F
:1002E000771F881FBB1F621773078407BA0720F0A8
:1002F000621B730B840BBA0BEE1F88F7E095089511
:1003000004D06894B111B5C0089598D088F09F5773
:1003100090F0B92F9927B751A0F0D1F0660F771F51
:10032000881F991F1AF0BA95C9F712C0B13081F031
:100330009FD0B1E008959CC0672F782F8827B85FC1
:1003400039F0B93FCCF3869577956795B395D9F792
:100350003EF490958095709561957F4F8F4F9F4F9C
:100360000895E89409C097FB3EF4909580957095A8
:1003700061957F4F8F4F9F4F9923A9F0F92F96E9F1
:10038000BB279395F695879577956795B795F11166
:10039000F8CFFAF4BB0F11F460FF1BC06F5F7F4F03
:1003A0008F4F9F4F16C0882311F096E911C0772315
:1003B00021F09EE8872F762F05C0662371F096E81E
:1003C000862F70E060E02AF09A95660F771F881FED
:1003D000DAF7880F9695879597F9089597F99F67AB
:1003E00080E870E060E008959FEF80EC08950024BD
:1003F0000A941616170618060906089500240A948A
:1004000012161306140605060895092E0394000C0F
:1004100011F4882352F0BB0F40F4BF2B11F460FF9E
:1004200004C06F5F7F4F8F4F9F4F089557FD9058C7
:10043000440F551F59F05F3F71F04795880F97FBA8
:10044000991F61F09F3F79F0879508951216130662
:100450001406551FF2CF4695F1DF08C01616170691
:100460001806991FF1CF86957105610508940895C6
:10047000E894BB2766277727CB0197F90895AA1B35
:10048000BB1B51E107C0AA1FBB1FA617B70710F07F
:10049000A61BB70B881F991F5A95A9F780959095B1
:0A04A000BC01CD010895F894FFCFD0
:00000001FF
